:020000023000CC
:10E000000D949AF00D94C3F00D94C3F00D94C3F0E9
:10E010000D94C3F00D94C3F00D94C3F00D94C3F0B0
:10E020000D94C3F00D94C3F00D94C3F00D94C3F0A0
:10E030000D94C3F00D94C3F00D94C3F00D94C3F090
:10E040000D94C3F00D94C3F00D94C3F00D94C3F080
:10E050000D94C3F00D94C3F00D94C3F00D94C3F070
:10E060000D94C3F00D94C3F00D94C3F00D94C3F060
:10E070000D94C3F00D94C3F00D94C3F00D94C3F050
:10E080000D94C3F00D94C3F00D94C3F00D94C3F040
:10E090000D94C3F00D94C3F00D94C3F00D94C3F030
:10E0A0000D94C3F00D94C3F00D94C3F00D94C3F020
:10E0B0000D94C3F00D94C3F00D94C3F00D94C3F010
:10E0C0000D94C3F00D94C3F00D94C3F00D94C3F000
:10E0D0000D94C3F00D94C3F00D94C3F00D94C3F0F0
:10E0E0000D94C3F00D94C3F00D94C3F00D94C3F0E0
:10E0F0000D94C3F00D94C3F00D94C3F00D94C3F0D0
:10E100000D94C3F00D94C3F00D94C3F00D94C3F0BF
:10E110000D94C3F00D94C3F00D94C3F00D94C3F0AF
:10E120000D94C3F00D94C3F00D94C3F00D94C3F09F
:10E130000D94C3F011241FBECFEFD1E8DEBFCDBFD9
:10E1400001E00CBF12E0A0E0B2E0ECE4F8EE03E086
:10E150000BBF02C007900D92A430B107D9F722E09F
:10E16000A4E0B2E001C01D92A630B207E1F70F941F
:10E17000E0F00D9424F401E80EBF0FEF0DBF112461
:10E180001FBE0D94E0F00D9400F08093C6008091C6
:10E19000C00086FFFCCF8091C00080648093C000E7
:10E1A000089520E030E02817390749F0EFECF7E058
:10E1B0003197F1F700C000002F5F3F4FF4CF089573
:10E1C000CF93DF93CDB7DEB7C052D1400FB6F894EE
:10E1D000DEBF0FBECDBF80E880936100109261006A
:10E1E00001E80EBF0FEF0DBF84B78EBBF894A89562
:10E1F00014BE80916000886180936000109260007E
:10E2000078946C9A749A22981092C0001092C1006F
:10E210008091C6008091C00082608093C00090E130
:10E220009093C40088E18093C1008091C000826017
:10E230008093C0009093C40000008CB100E010E017
:10E24000C12CD12C760197EC892E9BE1992EA12C23
:10E25000B12C20E1722E8091C00087FD26C00115EF
:10E26000110519F525E02A95F1F700004FEFC41AC2
:10E27000D40AE40AF40A91E080E0E1E6CE16EAEE80
:10E28000DE06E104F10408F490E0092F182FC7011D
:10E29000B601A50194010F94EDF3672B682B692B50
:10E2A000D1F68EB187258EB9D6CF0F5F1F4F0130C3
:10E2B000110509F075C2C25EDE4F1882CE51D14001
:10E2C000D12C212C312C812C912C5401412C512CFE
:10E2D000320120E030E080E001301105C1F041E082
:10E2E00052E16AE770E09091C00097FD10C0415084
:10E2F000510961097109B9F76BBFFA01479156914C
:10E300004F3F5F4F61F3EE27FF270994E8CF9091CD
:10E31000C600833001F120F4813071F038F014C070
:10E32000853029F1E0F0863099F135C09B3109F450
:10E330004BC200E010E0D0CFD926C25EDE4F9883FA
:10E34000CE51D14082E0F5CF292F30E0322F222765
:10E35000D92683E0EECF292BD92684E0EACF9E3060
:10E3600009F036C2D926212C312C85E0E2CFA1015B
:10E370004F5F5F4FE1E0F0E0EC0FFD1FE20DF31D9A
:10E380009083D9262417350709F424C21A01D1CF66
:10E390009D111EC202C0873061F62981233109F424
:10E3A000D7C058F5263009F4C5C0F8F42230E9F199
:10E3B000233009F467C0213009F0A0C11A8288E037
:10E3C0008B8381E48C8386E58D8382E58E8389E46B
:10E3D0008F8383E5888780E589878FE58A8782E355
:10E3E0008B87C12C0BE010E08EC1213109F457C09E
:10E3F00008F098C02031C9F081C1283109F46BC000
:10E4000048F4253109F4A4C008F427C1263109F4E1
:10E4100024C174C12A3109F451C008F471C02B31F0
:10E4200009F441C02D3119F069C1C12C3AC09D8158
:10E43000903339F48F818823B1F08130B1F488EAC8
:10E4400017C0892F807599F0903521F489E0E0E0BC
:10E45000F0E005C0983559F4E3E0F0E089E08093FE
:10E460005700849105C08EE103C082E001C080E0C6
:10E470001A821B829C831D828E831F82C12C07E01F
:10E4800010E041C1EA81E059E33028F4F0E0E050C7
:10E49000FE4F808101C080E01A828B833FC0CC2474
:10E4A000C3941A822EC18D81882321F0813021F4FA
:10E4B00088EA24C08EE122C082E020C01A82E1E016
:10E4C000F0E089E08093570084918B831C82C12CFB
:10E4D00004E010E018C18B81803551F48C818830C4
:10E4E00019F4E2E0F0E006C089E0E0E0F0E003C00B
:10E4F000E3E0F0E089E08093570084911A82E5CF51
:10E500008D81836C99E0E1E0F0E0082E9093570054
:10E51000E89507B600FCFDCF1A821B82C12C03E0F0
:10E5200010E0F1C01A82C12C02E010E0812C912C85
:10E530005401E9C06A817B818C819D810F940FF425
:10E540002B013C01440C551C661C771C1A82D8C058
:10E55000EA80FB80FE24EF24FE24233109F046C02C
:10E560008114F0EC9F06F3E0AF06B10470F423E0F1
:10E57000F401A0925B0020935700E89507B600FCD9
:10E58000FDCF4FEF941AA40AB40A8B85DE011196D1
:10E59000930182011B964C911B9790E0942B41E0D4
:10E5A0000C01F80120935B0040935700E89511247B
:10E5B0000E5F1F4F2F4F3F4F82E0E81AF10812966F
:10E5C000E114F10421F01A968C911A97E3CF95E0AB
:10E5D000F20160925B0090935700E89507B600FC4B
:10E5E000FDCF81E180935700E89533C0D301C2018C
:10E5F000B695A795979587956C01FE013B96C15EF0
:10E60000DE4FF983E883CF51D14000E010E00E15D2
:10E610001F05A9F0C15EDE4FE881F981CF51D140DD
:10E620006191C15EDE4FF983E883CF51D140C801CB
:10E630008C0D9D1D0F9416F40F5F1F4FE8CF20E047
:10E6400030E0000F111F221F331F040D151D261D62
:10E65000371D1A822801390153C08A819B8198276E
:10E66000892798278C010D5F1F4F1A822431C1F42E
:10E67000DE0111966BBEF2012791369112962C9312
:10E680001297FD01349613963C93139722E0420EA5
:10E69000511C611C711C02971296009759F72BC0F0
:10E6A000FE0131969F01280F391FB301A20141BD20
:10E6B000C52ED62EE72EFF24C2BC4F5F5F4F6F4F93
:10E6C0007F4FF89AA0B5A28331962E173F0779F7AE
:10E6D000AC014150510960E070E04F5F5F4F6F4FF8
:10E6E0007F4F440E551E661E771EE3E0F0E0EC0FF0
:10E6F000FD1FE80FF91F1082C12C05C080EC8A8332
:10E70000C12C02E010E08BE10F94C5F0C25EDE4F39
:10E710008881CE51D1400F94C5F0812F0F94C5F060
:10E72000802F0F94C5F085E1C25EDE4FD880CE51B8
:10E73000D140D826D0268EE00F94C5F0D126CE0148
:10E7400001967C01080F191F0E151F0591F0F701A6
:10E7500021917F01C15EDE4F2883CF51D140822FAE
:10E760000F94C5F0C15EDE4F4881CF51D140D42611
:10E77000EBCF8D2D0F94C5F0C25EDE4F8881CE5158
:10E78000D1408F5FC25EDE4F8883CE51D1409EB1B3
:10E7900080E189278EB900E010E0CC2009F499CD02
:10E7A0006C98749884E690E00F94D1F0000080910A
:10E7B000C0008D7F8093C00081E180935700E89571
:10E7C000EE27FF270994FFCF8BE1D82E81E0B1CD52
:10E7D00080E0AFCD190186E0ACCDA1E21A2EAA1BD4
:10E7E000BB1BFD010DC0AA1FBB1FEE1FFF1FA21701
:10E7F000B307E407F50720F0A21BB30BE40BF50BFE
:10E80000661F771F881F991F1A9469F76095709586
:10E81000809590959B01AC01BD01CF0108956927BA
:10E82000962769277827872778270895262FF9992B
:10E83000FECF1FBA92BD81BD20BD0FB6F894FA9AE3
:0CE84000F99A0FBE01960895F894FFCFDE
:04E84C000F020A00AD
:040000033000E000E9
:00000001FF
